:020000040000FA
:1000000087EF0AF012000100AC150000000F00009D
:100010005400000046EC05F0FB0EDBCFF3FFDB06DF
:10002000F35000090AE094EC05F0FA0EFFEC05F03D
:10003000F3E1151CF1E1010E01D0000E75EF05F0A2
:1000400046EC05F03B0EE12402E3E168E652E16E86
:10005000010EDB6A020EDB6AF90EDBCFF6FFFA0E49
:10006000DBCFF7FFFB0EDBCFF8FF0800F550DF6EAC
:10007000DF5002E199EF04F0250EDF5C02E08CEF27
:1000800004F0030EDB6A040EDB6A050EDB6A060E63
:10009000DB6A070EDB6AAEEC04F02D0EDF5C0CE0D1
:1000A0002B0EDF5C09E0200EDF5C06E0230EDF5C38
:1000B00003E0300EDF5C1AE1DF50300A14E0130A6F
:1000C0000FE0030A0AE00B0A05E0060AE4E1030E6A
:1000D000DB80E1D7030EDB82DED7030EDB84DBD7C8
:1000E000030EDB86D8D7030EDB88D5D72A0EDF5C5C
:1000F0001BE1AAEC04F0F8EC04F010E0030EDB8046
:1001000008680968130EDBCF0DF0140EDBCF0EF07C
:10011000FDEC09F0040E06C0DBFF03D0130EE1EC8A
:1001200004F0AEEC04F00BD0090EDB6A4FEC05F0E6
:1001300003E0C3EC05F0FAD7090EE1EC04F0030E7E
:10014000DBB0DB982E0EDF5C1BE1AEEC04F02A0E78
:10015000DF5C0BE1AAEC04F0F8EC04F003E1130E11
:1001600033EC05F0AEEC04F00BD0090EDB6A4FEC7B
:1001700005F003E0C3EC05F0FAD7090E33EC05F007
:10018000680EDF5C07E1AEEC04F0680EDF5C1DE199
:10019000030E18D0740EDF5C17E07A0EDF5C14E0FB
:1001A000480EDF5C06E0540EDF5C03E05A0EDF5CB5
:1001B00002E1020E07D06C0EDF5C03E06A0EDF5C2A
:1001C00004E1010E86EC05F0C9DBDF506E0A01E1A7
:1001D0007FD31E0A01E192D1200A01E18FD13F0AAB
:1001E00001E149D11A0A01E146D10D0A01E143D1E9
:1001F000200A01E140D13A0A01E13DD1200A01E1A2
:100200003AD1260A01E135D10D0A01E132D11A0AAB
:1002100001E1D9D0200A4AE0300A1FE0460A0EE088
:10022000250A01E083D3D950F90FE96EFF0EDA20D9
:10023000EA6E010EEE5E000EEE5AEE5A94EC05F0F8
:10024000250EE66E95DB03E1151C01E169D390EC08
:1002500005F001E26BD3DB2A69D3080EDB6A040EDA
:10026000DB50010806E2040EDB0458EC05F0DB501D
:100270008BDB080EDB5009E0030EDB50010B05E1C0
:1002800072DB01E04DD3080EDB6A64DBEFCFDFFFEA
:1002900008EC06F003E1151C01E142D390EC05F0F7
:1002A00001E3DB2A60DB01E141D33AD3070EDB50E7
:1002B00002080FE1D4EC05F0030E9BEC05F00E0EE6
:1002C000EECFDBFF0F0EEECFDBFF100EEECFDBFF2E
:1002D00020D0F70EDBCF17F0F80EDBCF18F0020EB0
:1002E000175E000E185AF70E17C0DBFFF80E18C085
:1002F000DBFF17C0E9FF18C0EAFF8BEC05F0166AB8
:100300000E0E14C0DBFF0F0E15C0DBFF100E16C063
:10031000DBFF0E0EDBCFE6FF0F0EDBCFE6FF100E8E
:10032000DBCFE6FFD8EC09F0E552E552E552130EBB
:1003300007C0DBFF140E08C0DBFF060EDB5005E034
:10034000130ECFEC05F001E26ADBF3EC05F002E2FC
:10035000130E37DBB6EC05F006E0040ECFEC05F02B
:1003600002E2050E2EDB030EDBB005D0FCDA01E065
:10037000D7D2080EDB6A090EDB6A0E0EDBCFF6FF62
:100380000F0EDBCFF7FF100EDBCFF8FF0800F550A4
:10039000DF6EDF5014E0F9EC05F011E208EC06F036
:1003A00003E1151C01E1BCD2BBDB01E3DB2A090E32
:1003B000DB2AD9500E0FE96E000ECBDBE7D7D3DA7C
:1003C00001E1B4D2ADD2C6DA110EEECFDBFF120ED0
:1003D000EDCFDBFF110EDBCFE6FF120EDBCFE6FF2A
:1003E000CAEC09F0E552E552130EF3CFDBFF140E11
:1003F000F4CFDBFF060EDB5004E0130ED0DB01E28E
:100400000EDBF3EC05F002E2130EDBDAAFDB05E006
:10041000040EC5DB02E2050ED4DA030EDBB005D014
:10042000A2DA01E07DD2080EDB6A090EDB6A110E4A
:10043000DBCFE9FF120EDBCFEAFFEFCFDFFFDF50AC
:1004400014E0D7DB12E2E4DB03E1151C01E168D222
:1004500067DB01E3DB2A090EDB2A110EDB2ADBCF87
:10046000E9FF120EE8E3DB2AE6D77DDA01E15ED28E
:1004700057D2030EDB8E070EDB0410E195DB040E72
:100480005ADB0A0EEECFDBFF0B0EEECFDBFF0C0EBE
:10049000EECFDBFF0D0EEECFDBFF6CD0070EDB5097
:1004A00003082CE1030EDBAE0DD0B2DA020E76DAD1
:1004B000EFCF14F0156A166A176A14AE39D01568B2
:1004C000166835D0F70EDBCF15F0F80EDBCF16F03F
:1004D000020E155E000E165AF70E15C0DBFFF80E61
:1004E00016C0DBFF15C0E9FF16C0EAFFEFCF14F01E
:1004F0000A0E14C0DBFF0B0EDB6A38D0070EDB5090
:10050000020809E1030EDBAE04D059DB16AE10D0B1
:100510000ED055DB0DD0030EDBAE12D079DA020E11
:100520003DDAF9DA166A176A15AE02D0166817684E
:10053000E2DA0C0E16C0DBFF0D0E17C0DBFF1AD07F
:10054000F70EDBCF16F0F80EDBCF17F0020E165EBB
:10055000000E175AF70E16C0DBFFF80E17C0DBFFB0
:1005600016C0E9FF17C0EAFFD6DAC5DA0C0EDB6A5F
:100570000D0EDB6A060EDB5005E1010EF36E050E73
:10058000F3CFDBFF150EDB6A160EDB6AD950370F8F
:10059000146E000EDA20156E390E14C0DBFF3A0E11
:1005A00015C0DBFF380EDB6A080EDB6A0A0EAEDA16
:1005B000DF50780A12E0200A10E0280A0CE0200A36
:1005C0000AE03F0A06E00D0A02E0200A08E1020EF6
:1005D00005D0080E03D0080EDF26100E97DA030EA2
:1005E000DBBE02D0DB92DB94DB50800B24E08ADAA6
:1005F000D890030EEB50000A08E6000EEE5C000EE9
:10060000EE58000EEE58000EEE5815E213DA0B68A5
:100610000C680D680E6892EC09F00A0E02C0DBFF50
:100620000B0E03C0DBFF0C0E04C0DBFF0D0E05C07C
:10063000DBFF2D0E08D0030EDBA202D02B0E03D061
:10064000DBA408D0200EF36E170EF3CFDBFF150EE0
:10065000DB2A02D0170EDB6A050EDB5003E1B7D9A7
:1006600001E189D0880E146E150E156E000E166EFF
:10067000070EDBCF17F0186A196A1A6A17C00BF059
:1006800018C00CF019C00DF01AC00EF0D3D92AEC26
:100690000AF014500224F36E15500320F46E165025
:1006A0000420F86EF4CFF7FFF3CFF6FF0800090E31
:1006B000F5CFDBFF580EDF5C0FE1610EF36E090E24
:1006C0007BD90AE3200E146E090EDBCFE7FF14502E
:1006D000E75E090EE7CFDBFF070EDBCF14F0156AEC
:1006E000166A176A0FDA14C00BF015C00CF016C0AA
:1006F0000DF017C00EF0EECF06F0EECF07F0EECF04
:1007000008F0EFCF09F02AEC0AF009C0EDFF08C0AD
:10071000EDFF07C0EDFF06C0EFFF390EDBCFE9FFAD
:10072000DB063A0EDBCFEAFF01E2DB06090EDBCF88
:10073000EFFF150EDB2A4BD995E1030EDBA61DD08A
:100740006F0EDF5C06E1C1D918E3150EDB285BDA1A
:1007500014D0780EDF5C09E0580EDF5C06E0620E14
:10076000DF5C03E0420EDF5C08E1020EF36E160E62
:10077000F3CFDBFF02D0150EDB6A030EDB50100B4C
:100780000EE0040EDBCF14F0050EDB50D8801454BD
:1007900006E2060EDB5003E1040EDB5034DA95D995
:1007A0000AE2050EDBCFE7FF150EDB50E75E050E14
:1007B000E7CFDBFF02D0050EDB6A040EDBCF14F0BF
:1007C000160E45D9D880145414E2160EDBCFE6FF7E
:1007D000150EDBCFE6FF040EDBCFE6FF050EDB5088
:1007E000E552E75CE552D880E754E552D880E754FB
:1007F0005FD9030EDB50010B0BE1080EDB5008E064
:10080000B2D801E08DD0080EDB50BED8080EDB6AEE
:10081000170EDB5007E088D9170EF1D903E1151C3C
:1008200001E17ED0160EDB5016E07ED9300EE66E6A
:100830009FD802E1151C74E077D9DFCFE6FF50ECBA
:1008400009F0E552E552E552F4CF15F00001F31C32
:1008500002E1151C65E0050EDBCF14F0160EDB502F
:10086000D880145409E2050EDBCFE7FF160EDB50EB
:10087000E75E050EE7CFDBFF300EE66E050ECBD947
:100880004FE1390EDB2ADBCFE9FF3A0E01E3DB2A29
:10089000DBCFEAFF090EEFCFDBFFDB500EE044D9E0
:1008A000090EADD902E1151C3BE0390EDB2ADBCF86
:1008B000E9FF3A0EEDE3DB2AEBD755D831E1160E0E
:1008C000DBCFE6FF080EC3D8E552E7245DD82ED073
:1008D000070EDB50030A1CE0010A14E0030A07E0DC
:1008E0007BD9DBCFEEFF020EDBCFEDFF1FD0F5D8BB
:1008F000196A17AE02D0186819682CD8BCD819C06C
:10090000EEFF14D0EAD817BE186824D8B4D80ED099
:1009100063D9DBCFEFFF0AD07BD905E1151C03E1DA
:10092000F368F46810D0FCD801E3DB2A79D935EFFD
:1009300000F0010EDBCF14F0020EDBCF15F014C077
:10094000F3FF15C0F4FF3B0EE15C02E2E16AE55201
:10095000E16ECBD029D9020E9BEF05F061D90800DA
:10096000F550DF6E1200200EE66E080E0BEF06F05B
:1009700050EC09F0E552E552E552F3CF14F0F4CF14
:1009800015F00001F31C1200146E156AD950010F06
:100990004DD91450EE261550ED221200185E000EAF
:1009A000195AF70E18C0DBFFF80E19C0DBFF18C08C
:1009B000E9FF19C0EAFF1200DBCFF4FFF350F45C4B
:1009C0001200DB50E76E040EE7CFDBFF12000A0EC9
:1009D000DBCF14F00B0EDBCF15F00C0EDBCF16F0D7
:1009E0000D0EDBCF17F01450151016101710120053
:1009F000130EEECFDBFF140EEDCFDBFF130EDBCFBC
:100A000014F0140EDBCF15F00001800E1514120047
:100A1000F70EDBCF18F0F80EDBCF19F01200050E41
:100A2000DB50E66ED950130F01D9E552E750EE6E58
:100A3000ED6A12000A0EDBCF06F00B0EDBCF07F0DB
:100A40000C0EDBCF08F00D0EDBCF09F01200DBCF70
:100A5000E6FF150EDBCFE6FF050EDB50E552E7247F
:100A6000E552E7241200DB50CED8010EF36E060EDD
:100A7000F3CFDBFF1200EE50EFCFEAFFE96E16C0B6
:100A8000EEFF17C0EEFF18C0EEFF1200D9CFE6FF51
:100A9000DACFE6FFE1CFD9FFE2CFDAFF1200DFCFF6
:100AA000E6FFE66A65EC0AF0E552E552F350120003
:100AB000E76E080EE7CFDBFF1200EECF14F0EECFAB
:100AC00015F0EFCF16F0176A1200050EDBCF14F009
:100AD000150EDB50D88014541200010EDBCF16F037
:100AE000020EDBCF17F0186A1200E552E5CFDAFFED
:100AF000E7CFD9FF12000A0E14C0DBFF0B0E15C0A2
:100B0000DBFF1200D9500A0F16EF06F0F36E070E46
:100B1000F3CFDBFF1200EECF14F0EFCF15F0120091
:100B2000010EDB2A020E1200FC0EDBCFE6FFFD0EEB
:100B3000DBCFE6FF1200145E000E155AF70E14C04C
:100B4000DBFFF80E15C0DBFF14C0E9FF15C0EAFF9C
:100B50001200DA20EA6EEF2AEECFF6FF000EEF2247
:100B6000EECFF7FFEF22EECFF8FF1200040EDBCF3F
:100B7000E6FF130EDB50E552E75C9ADFDB5004DF43
:100B8000060EDB501200090EDB500A0DF350DF2475
:100B9000D00FE76E090EE7CFDBFFAEEF04F0DB50BE
:100BA000F36E050EDCEF04F0F70EDBCF14F0F80E59
:100BB000DBCF15F01200DFCFE6FFB8EF04F028DF3F
:100BC000030EECDE5DEF05F00AEC00F0E552E552B5
:100BD000E552E55200091200BDDEEE50EFCFEAFF0C
:100BE000E96E010E1200130EDB50F36E040EDCEF03
:100BF00004F0040EDB50F36E090EDCEF04F0DBCFE3
:100C0000E6FFB8EF04F0E76E050EE7CFDBFF12005A
:100C10008BDFDBEF05F0DBCFE6FF86DFE4EF05F0EF
:100C2000D950F90FE96EFF0EA9EF05F0E96E000E3D
:100C3000DA20EA6E12000F0E9316811693949396A3
:100C40008194819620D90F0E8116300E811227D8FB
:100C50003FD90F0E8116300E811221D839D90F0ECF
:100C60008116300E81121BD833D90F0E8116818A5E
:100C700016D8280EE66E17D8E552080EE66E13D881
:100C8000E552010EE66E0FD8E552060EE66E0BD861
:100C9000E5520F0EE66E07D8E55200D012008186AD
:100CA0003CD981961200D9CFE6FFE1CFD9FF39D9DF
:100CB000819481960F0E8116FE0EDBCF14F0F00E9C
:100CC00014148112ECDF0F0E8116FE0EDB50146E31
:100CD000156A040ED89014361536E804FBE1F00EC0
:100CE00014148112DCDF00D0E552E7CFD9FF1200E7
:100CF000D9CFE6FFE1CFD9FF14D9818481960F0EB9
:100D00008116FE0EDBCF14F0F00E141481128186D2
:100D100004D981960F0E8116FE0EDB50146E156AF3
:100D2000040ED89014361536E804FBE1F00E1414C6
:100D300081128186F2D8819600D0E552E7CFD9FFA3
:100D40001200D9CFE6FFE1CFD9FFFD0EDBCFF6FFD2
:100D5000FE0EDBCFF7FF0800F550146E156A145035
:100D6000151011E0FD0EDBCFF6FFFE0EDBCFF7FF17
:100D70000800F550E66EBCDFE552FD0EDB2AFE0EE4
:100D800001E3DB2AE2D700D0E552E7CFD9FF12001A
:100D9000D9CFE6FFE1CFD9FFFD0EDBCFE9FFFE0E95
:100DA000DBCFEAFFEF50146E156A1450151010E0F7
:100DB000FD0EDBCFE9FFFE0EDBCFEAFFEF50E66E64
:100DC00097DFE552FD0EDB2AFE0E01E3DB2AE4D7B6
:100DD00000D0E552E7CFD9FF1200D9CFE6FFE1CF2F
:100DE000D9FFE652FE0EDB50146E156A010E141880
:100DF00001E1155006E1FD0EDBCF14F0800E142446
:100E0000DF6EFE0EDB50146E156A020E141801E13F
:100E1000155006E1FD0EDBCF14F0C00E1424DF6E7A
:100E2000DF50E66E40DFE552E552E552E7CFD9FFED
:100E30001200D9CFE6FFE1CFD9FFE652E66AFE0EF7
:100E4000DB50E66ECADFE552E552DF6ADF50146E12
:100E5000156AD890155004E6100E145C000E155853
:100E600006E2200EE66E44DFE552DF2AEFD7E66A9F
:100E7000FE0EDB50E66EB1DFE552E552E552E5527B
:100E8000E7CFD9FF1200D9CFE6FFE1CFD9FF020E9D
:100E9000E126DE6ADD6ADECF14F0DDCF15F0D890F2
:100EA000155004E6100E145C270E155806E20000DB
:100EB000DF2A010E01E3DB2AEED700D0020EE15C4F
:100EC00002E2E16AE552E16EE552E7CFD9FF120096
:100ED000D9CFE6FFE1CFD9FF020EE126DE6ADD6A57
:100EE000DECF14F0DDCF15F0D890155004E6C40E17
:100EF000145C090E155806E20000DF2A010E01E31A
:100F0000DB2AEED700D0020EE15C02E2E16AE55294
:100F1000E16EE552E7CFD9FF1200000000000000AB
:100F20001200D9CFE6FFE1CFD9FF020EE126DE6A3B
:100F3000DD6ADECF14F0DDCF15F0D890155004E651
:100F4000E80E145C030E155806E20000DF2A010EBD
:100F500001E3DB2AEED700D0020EE15C02E2E16A97
:100F6000E552E16EE552E7CFD9FF1200D9CFE6FF97
:100F7000E1CFD9FF020EE126FD0EDBCF14F0FE0E0D
:100F8000DBCF15F0D89014361536D89014361536B8
:100F9000010E1424C26E0A0EE66EB0EC0AF0E552A1
:100FA000D2EC0AF0CDEC0AF0000901E0FBD7BBEC73
:100FB0000AF0F3CFDEFFF4CFDDFFDECF14F0DDCF9C
:100FC00015F014C0F3FF15C0F4FF020EE15C03E25C
:100FD00000D0E16AE552E16EE552E7CFD9FF120099
:100FE0008168936A7F6AF19E7C687E6A7E807E82D9
:100FF000896A0F0E926E806A8268BF0E946E94802A
:101000009482948494869488948A949C948ED08EAE
:10101000D09C786A1200C280C19AC198C08EC08AE2
:10102000C088C096C084C092C0801200D9DFF3DFB0
:101030008998FA0EE66E4EEC0AF0E5528988FBDDDF
:10104000010EE66EF6DEE552560EE66E150EE66E03
:1010500078DEE552E552FA0EE66E4EEC0AF0E55205
:10106000020EE66EE6DEE552480EE66E41DEE55221
:10107000450EE66E3DDEE5524C0EE66E39DEE5527B
:101080004C0EE66E35DEE5524C0EE66E31DEE55274
:101090004F0EE66E2DDEE552FA0EE66E4EEC0AF0CD
:1010A000E552020EE66EC5DEE5524B0EE66E150EFB
:1010B000E66E47DEE552E5528950100B01E0010E65
:1010C000166E176A1650171002E0000E01D0010EBE
:1010D000146E156A1450E8B08988E8A08998000E4B
:1010E000E66EE66A43DFE552E552F3CF96F0F4CFC1
:1010F00097F096C0E6FF97C0E6FF460E146E150EF9
:10110000156E166A14C0E6FF15C0E6FF16C0E6FFAE
:1011100052CFE6FF53CFE6FFABEC08F0176E070E99
:10112000E15E1750F3CF64F0F4CF65F00B0EE66E7E
:10113000020EE66E52DEE552E55252CFE6FF53CF85
:10114000E6FF26DEE552E552960EE66E4EEC0AF01C
:10115000E552B2D71200D9CFE6FFDACFE6FFE1CFF2
:10116000D9FFE2CFDAFFE652E652E652E652D95014
:10117000F90F146EFF0EDA20156E020E14C0DBFF9D
:10118000030E15C0DBFF020EDBCFE6FF030EDBCF45
:10119000E6FFF90EDBCFE6FFFA0EDBCFE6FFFB0E34
:1011A000DBCFE6FFD950FC0FE66EFF0EDA20E66ECD
:1011B00020EC00F0146E070EE15C02E2E16AE552F9
:1011C000E16E1450F3CFDEFFF4CFDDFFFC0EDBCF7A
:1011D000E9FFFD0EDBCFEAFFEF6ADECF14F0DDCFD3
:1011E00015F014C0F3FF15C0F4FF040EE15C02E239
:1011F000E16AE552E16EE552E5CFDAFFE7CFD9FFCC
:101200001200060EF66E000EF76E000EF86E0F015D
:101210000900F550596F0900F5505A6F03E15967FD
:1012200001D03DD00900F550546F0900F550556FBD
:101230000900F550566F09000900F550E96E0900E4
:10124000F550EA6E090009000900F550576F0900D2
:10125000F550586F09000900F6CF5BFFF7CF5CFF30
:10126000F8CF5DFF54CFF6FF55CFF7FF56CFF8FF0D
:101270000F01575302E1585307E00900F550EE6E95
:101280005707F8E25807F9D75BCFF6FF5CCFF7FFB7
:101290005DCFF8FF0F015907000E5A5BBFD7120050
:1012A000D9CFE6FFDACFE6FFE1CFD9FFE2CFDAFF11
:1012B000FB0EDBCF14F0FC0EDBCF15F00001800E2F
:1012C00015141AE1FB0EDBCFE9FFFC0EDBCFEAFFC2
:1012D000EECFF3FFEDCFF4FFEE2A000EEF22F3CFB7
:1012E000E9FFF4CFEAFFFD0EDBCFEFFFEF50156A09
:1012F000F36E15C0F4FF10D0FB0EDB50FE0806E1C4
:10130000FD0EDBCFE6FF95EC0AF005D0FD0EDBCF3E
:10131000E6FFD4EC0AF0E552E552E5CFDAFFE7CF7D
:10132000D9FF120006500B02F3CF02F0F4CF03F006
:101330000C02F3500326000EF420046E06500D023A
:10134000F3500426000EF420056E06500E02F350F2
:10135000052607500B02F3500326F4500422000E1A
:10136000052207500C02F3500426F45005220750C2
:101370000D02F350052608500B02F3500426F450DA
:10138000052208500C02F350052609500B02F350B9
:1013900005261200FE0EE3CFE9FFFF0EE3CFEAFFC2
:1013A000F36AF46AEE5203E0F34AF42AFBD7120020
:1013B000FF0EE3CFF8FFE552FF0EE3CFF7FFE55254
:1013C000FF0EE3CFF6FFE552E66AE66AE66A090039
:1013D000F55209E0FD0EE32A05E1FE0EE32A02E1E3
:1013E000FF0EE32AF4D7FD0EE3CF07F0FE0EE3CFA6
:1013F00008F0FF0EE3CF09F0120009C013F008C097
:1014000012F008500D02F4CF07F0F3CF06F00950A8
:101410000E02F4CF09F0F3CF08F00D02F3500726C7
:10142000F4500822E86A092212500E02F3500726EF
:10143000F4500822E86A09220EAE23EF0AF0125097
:10144000085E1350095A13AE000C0D50085E0E5082
:10145000095A000C056A046A036A026A200EE76EE4
:10146000D890063607360836093602360336043673
:1014700005360B50025C0C5003580D5004580E50AA
:10148000055809E30B50025E0C50035A0D50045AE4
:101490000E50055A062AE72EE4D71200FF0EE3503D
:1014A0001C6EEF0E01D0F30EE76EE72E55EF0AF03B
:1014B0000C0E1B6EE76AE72E5BEF0AF01B2E5AEF4D
:1014C0000AF01C2E53EF0AF01200F36AF46AFF0EC2
:1014D000E124E96EFF0EE220EA6EED6607D02F0EE2
:1014E000EF6404D03A0EEF6001D0F32A1200600ED0
:1014F000F36E00EE00F00F0E01D81200EA6002D089
:10150000EE6AFCD7F350E9601200EE6AFCD71EEEDB
:1015100000F02EEE00F0F86A019C01EC09F0D5EC29
:101520000AF016EC08F0FBD71200FF0EE350ACBA3D
:1015300004D0AF6AAB8EAC8A949CACA2FED7AD6EE1
:10154000F36EF46A120025303464004D65737572D1
:10155000652043483000202053414C555420200042
:10156000FF0EE350E84E1200000000D000D000D083
:10157000E82EFAD71200C450176E166AC350161020
:10158000F36E17C0F4FF1200303132333435363782
:10159000383961626364656600FFC250020B01E086
:1015A000010E1200C28212001200120031323334D6
:1015B000353637383930313233343500000F505238
:1015C0004F4A455420433138203A31384632364B61
:1015D00032785F4C4344327831362E6D63700D00A3
:1015E00000000000000000000000000000000000FB
:1015F0000000000000000000000000000000120FCA
:10160000FFFFFFFFFFFFFFFFFFFFFFFFFFFFFFFFEA
:10161000FFFFFFFFFFFFFFFFFFFFFFFFFFFFFFFFDA
:10162000FFFFFFFFFFFFFFFFFFFFFFFFFFFFFFFFCA
:10163000FFFFFFFFFFFFFFFFFFFFFFFFFFFFFFFFBA
:0200000400F00A
:020000040030CA
:0E0000000002191E008980000FC00FE00F40A3
:020000040020DA
:08000000FFFFFFFFFFFFFFFF00
:00000001FF
